:1000000032EF0DF06896000C046ED8CF05F0E0CF0B
:1000100006F00001E9CF0CF0EACF07F0E1CF08F0DD
:10002000E2CF09F0D9CF0AF0DACF0BF0F3CF12F01C
:10003000F4CF13F0FACF14F0F5CF15F0F6CF16F099
:10004000F7CF17F000C00EF001C00FF002C010F0A3
:1000500003C011F0F2AA30EF00F0F2B421EF01F08A
:10006000A0AA36EF00F0A1BAE5EF07F00EC000F04D
:100070000FC001F010C002F011C003F00CC0E9FF86
:1000800007C0EAFF078E08C0E1FF09C0E2FF0AC00F
:10009000D9FF0BC0DAFF12C0F3FF13C0F4FF14C086
:1000A000FAFF15C0F5FF16C0F6FF17C0F7FF0450A2
:1000B00006C0E0FF05C0D8FF1000F76ACA0FF66E51
:1000C000000EF7220900F5501200280C0106F76A0D
:1000D000DE0FF66E000EF7220900F5501200000345
:1000E00002FFFFFFFFFFFFFFFFFFFFFFFFFFF76ABA
:1000F000FE0FF66E000EF7220900F550120000FF09
:1001000002FFFFFFFFFFFFFFFFFFFFFFFFFFF76A99
:100110001E0FF66E010EF7220900F5501200400086
:100120000800400000000000000000000000000087
:100130000000000000000000000000000000F76A5E
:100140004E0FF66E010EF7220900F5501200400026
:10015000000040000000000000000000000000005F
:100160000000000000000000000000000000F76A2E
:100170007E0FF66E010EF7220900F55012000902FB
:100180004300020100803209040000010202010064
:1001900005240010010424020205240600010524A0
:1001A000010001070581030800FA09040100020AA1
:1001B000000000070502024000010705820240001E
:1001C0000100F76AD20FF66E010EF7220900F55012
:1001D00012000200F76AE40FF66E010EF722090022
:1001E000F550120012171B20FFFFFFFFF76AFC0FEC
:1001F000F66E010EF7220900F550120012011001EF
:100200000200004061043300000101020001F76AAE
:100210001E0FF66E020EF7220900F55012000403BD
:10022000090408034300430053001803530045002A
:100230005200490041004C002000440045004D00A0
:100240004F00010E2A26D8B02B2AD8B42C2AD8B4B5
:100250002D2AF29436EF00F06D92699468A402D0D2
:100260006894FCD7F1EF07F0400E0401016F040E13
:10027000036F180E026F880E006F046B040E076F79
:10028000580E066F0001000C70A002D0EDDF7090D8
:10029000689AFAEF07F06A6A689200EF08F0D9915D
:1002A000D8BFD981D89FD851100803E2000E016E43
:1002B00017D0D9A10BD0036AD85109DFFF0802E19A
:1002C000000E01D0010E016E0BD00AD0036AD85186
:1002D0000EDFFF0802E1000E01D0010E016E00D01A
:1002E000000CDD51DF03F3CF01F0F4CF00F0E003A9
:1002F000F3500026DE51DF03F3500020026E000CA5
:10030000036AD751700FE96E0F0E0320EA6EEF6A91
:10031000D7C0D8F0C4DF015222E0DE6BD7C0DDF0D9
:10032000E06B080EDF6FDDDF01C0E9FF040E022481
:10033000EA6EEF6ADE6BD7C0DDF0E06B080EDF6FB0
:10034000D0DF02C0D9F001C0D8F0040ED827000ECB
:10035000D923D8C0E9FF040ED925EA6EEF6A000C54
:10036000010ED66FD6510F0805E3D6C0D7F0C8DF0F
:10037000D62BF8D7000C446A436A250E426E800ED5
:10038000416E456A466A080E476E966B9591496ABA
:10039000486A916B9291000CCC6BCC5101080AE336
:1003A000036ACC513F0FE96E000E0320EA6EEF6A3C
:1003B000CC2BF3D7E0DF336A010E346E326A000CC7
:1003C0006A6A686A9F0E6B6E3D0E696E6E6AC8DF60
:1003D000E3DF160E706E68A602D014DEFCD76D98AF
:1003E00043DF030E3A6E06EF08F0698468986D8269
:1003F0000CEF08F0689C12EF08F0D1C03BF0000C45
:10040000FF0E3B6E000CCF6B3E5226E0CF513F08F3
:1004100023E3355005E0020A08E0010A0BE00FD0A3
:10042000036A3D50A4DED06F0AD0036A3D50EFDE70
:10043000D06F05D0036A3D50D9DED06F00D03D2A81
:100440003E06CF51CF2B580FE96E040EEA6ED8B09E
:10045000EA2AD0C0EFFFD8D73E5204E1CF5140087E
:1004600001E0326ACFC0D1F0C8DF000C3D6A356AC6
:1004700004011B51010A000107E0030A0AE0010A16
:100480000BE0220A1BE02BD0120E3E6E030E356EDF
:1004900028D0430E3E6E25D0020E356E036A04014D
:1004A0001A51360FE96E000E0320EA6EEFCF3DF0D1
:1004B000036A3D500001ABDE3E6E13D0036A0401B7
:1004C0001A51000187DE3D6E3D3C01D006D0036A23
:1004D0003D504DDE3E6E05D002D092DF0ED090DF53
:1004E0000CD004011F5305E13E501E5D02E21EC404
:1004F0003EF0010E326E000186DFA1EF03F0CE5315
:1005000004E1040E3A6E2CDFC9D0050E3A6E040EDB
:10051000D16F980ED06F010ECF6FCF510F08D8A0BA
:10052000BDD0CFC0D7F0ECDED26B036ACF51DFDD98
:10053000FF0859E0040ED26FD890CF35036AFFDD73
:100540000900F5CF03F0D36F03C0D4F0DE6BCFC04A
:10055000DDF0E06B080EDF6FC4DE01C0D6F0010EE7
:100560000124016E000E0220036E01C0E9FF040E9B
:100570000324EA6ED3C0EFFFDE6BCFC0DDF0E06B8B
:10058000080EDF6FAEDE01C0D6F0020E0124016E50
:10059000000E0220036E01C0E9FF040E0324EA6E80
:1005A000D1C0ECFFED52D0C0EFFFD890CF35036A39
:1005B000C6DD0900F5CF03F0D0270350D123880E04
:1005C000D56FD4B1D581D4B3D583DE6BCFC0DDF088
:1005D000E06B080EDF6F85DE01C0E9FF040E022428
:1005E000EA6ED5C0EFFF036ACF5171DDFF0840E02E
:1005F000D283DE6BCFC0DDF0E06B080EDF6F71DE03
:1006000002C0D7F001C0D6F0040ED627000ED723C3
:10061000020ED625016E000ED721036E01C0E9FF40
:10062000040E0324EA6ED1C0ECFFED52D0C0EFFF00
:10063000D890CF35036A6BDD0900F5CF03F0D027E2
:100640000350D123DE6BCFC0DDF0E06B080EDF6F0F
:1006500048DE02C0D7F001C0D6F0040ED627000E47
:10066000D723D6C0E9FF040ED725EA6E400EEF6E01
:10067000D251060802E10E0ED26F036ACF5127DD78
:100680000108D8A4D289036ACF51700FE96E0F0E0A
:100690000320EA6ED2C0EFFFCF2B3FD79BEF03F0D2
:1006A00004011951000A00010DE0010A14E0020AD8
:1006B0001EE0060A27E0030A2CE00E0A2CE0010ADD
:1006C00030E03DD034C058F40401596B020E0001F3
:1006D000D16F93DE36D004011A2D06D0010E3416E8
:1006E0000001D16B8ADE02D000018ADE2AD004012B
:1006F0001A2D05D034820001D16B7FDE02D00001BB
:100700007FDE1FD0020E326E1AC43CF0D16B75DE54
:1007100018D0ACD616D033C058F4010ED16F6DDEB0
:1007200010D004011A51010808E31AC433F01AC4A6
:10073000CEF00001E4D6D16B60DE000102D060DEB5
:1007400000D015EF05F033C0CEF004011951000AB6
:10075000000105E00A0A0BE0010A26E037D0040197
:10076000586B596B020E0001D16F47DE31D0CE536A
:1007700019E0010ECE5D036A24DD016E04011C5DEB
:10078000D8A002D000010ED0036A1C513F0FE96EC1
:10079000000E0320EA6EEFCF58F4010E0001D16F76
:1007A0002CDE01D02DDE14D0CE530EE0036A0401FE
:1007B0001C513F0FE96E000E0320EA6E1AC4EFFFD2
:1007C0000001D16B1ADE01D01BDE02D019DE00D091
:1007D00015EF05F0CF91CEBFCF81CE9FCFA117D01F
:1007E000DE6BCEC0DDF0E06B080EDF6F7ADD02C09D
:1007F000D1F001C0D0F0040ED027000ED123D0C01C
:10080000E9FF040ED125EA6E880EEF6E0DD0DE6B87
:10081000CEC0DDF0E06B080EDF6F63DD01C0E9FFE5
:10082000040E0224EA6EEF6A8AEF04F0CF91CEBF85
:10083000CF81CE9FCFA117D0DE6BCEC0DDF0E06BB5
:10084000080EDF6F4EDD02C0D1F001C0D0F0040E03
:10085000D027000ED123D0C0E9FF040ED125EA6EC7
:10086000840EEF6E0ED0DE6BCEC0DDF0E06B080EB6
:10087000DF6F37DD01C0E9FF040E0224EA6E840E4B
:10088000EF6E90EF04F0CF91CEBFCF81CE9FCFA17E
:1008900017D0DE6BCEC0DDF0E06B080EDF6F21DD20
:1008A00002C0D2F001C0D1F0040ED127000ED22335
:1008B000D1C0E9FF040ED225EA6EEFCFD0F00ED002
:1008C000DE6BCEC0DDF0E06B080EDF6F0ADD01C02D
:1008D000E9FF040E0224EA6EEFCFD0F0D0AF02D0D1
:1008E000D0B502D0000E01D0010E016E9AEF04F0D7
:1008F0001CC4D8F0D4DC015229E004011951010ACA
:10090000000105E0020A09E0030A0DE01DD01CC445
:10091000CEF060D7D16B71DD19D01CC4CEF086D774
:10092000D16B6BDD13D00401586B596B1CC4CEF036
:100930000001A9D7015204E0010E0401586F000123
:10094000020ED16F5ADD02D05BDD00D015EF05F04D
:10095000FE0E3B6E000C04011C2D01D002D01C5376
:1009600049E11951000A00010BE0010A0DE0210ADA
:100970001CE0010A1FE0030A2EE0010A31E037D033
:10098000010E986FE5DF35D0040EEA6E580EE96E61
:10099000E26A4A0EE16E080E016EE6CFEEFF012E0E
:1009A000FCD71EC4D1F029DD24D0020E986F9581AA
:1009B000CFDF1FD0040EEA6E580EE96EE26A410ED8
:1009C000E16E070E016EE6CFEEFF012EFCD7070E9B
:1009D000D16F13DD0ED01AC496F0D16B0EDD09D0A5
:1009E0001AC449F01BC448F0D16B07DD02D008DD02
:1009F00000D00401000115EF05F0326A040118511E
:100A00007F0B000A000107E0010A07E0030A07E084
:100A1000230A07E008D044D608D095D606D068D778
:100A200004D099D702D0ECDC00D03AEF07F0DE6BAF
:100A3000CFC0DDF0E06B080EDF6F53DC01C0E9FFD3
:100A4000040E0224EA6EEFCFD1F0D051020806E185
:100A5000D1AD02D0D06B02D0010ED06FD0510308BF
:100A600019E1840ED16FDE6BCFC0DDF0E06B080EB4
:100A7000DF6F37DC02C0D5F001C0D4F0040ED427FC
:100A8000000ED523D4C0E9FF040ED525EA6E840EEE
:100A9000EF6E07D0D02D03D0C80ED16F02D0880ED4
:100AA000D16FD890CF35036A9FEC00F00900F5CFE5
:100AB00003F0D26F03C0D3F0DE6BCFC0DDF0E06B8C
:100AC000080EDF6F0EDC01C0D4F0010E0124016EB0
:100AD000000E0220036E01C0E9FF040E0324EA6E3B
:100AE000D2C0EFFFD3B1D181D3B3D183DE6BCFC0FE
:100AF000DDF0E06B080EDF6F71EC01F001C0E9FF83
:100B0000040E0224EA6ED1C0EFFF000C036ADC5130
:100B1000700FE96E0F0E0320EA6EEF5219E0DE6BE4
:100B2000DCC0DDF0E06B080EDF6F71EC01F002C09D
:100B3000DEF001C0DDF0040EDD27000EDE23DDC097
:100B4000E9FF040EDE25EA6EEFCFDDF0DDAF02D067
:100B5000000E01D0010E016E000CD7C0DCF0D6DF14
:100B60000152D8B47CD0DE6BD7C0DDF0E06B080E4C
:100B7000DF6F71EC01F002C0DDF001C0DCF0040EAB
:100B8000DC27000EDD23010EDC25016E000EDD21C9
:100B9000036E01C0E9FF040E0324EA6ED8C0EFFF24
:100BA000DA5102081EE1DE6BD7C0DDF0E06B080E03
:100BB000DF6F71EC01F002C0DDF001C0DCF0040E6B
:100BC000DC27000EDD23DCC0E9FF040EDD25EA6E24
:100BD000EFCFDBF0DBAD02D0DA6B02D0010EDA6FC3
:100BE00018D0DA51040815E1DE6BD7C0DDF0E06BF8
:100BF000080EDF6F71EC01F001C0E9FF040E022462
:100C0000EA6EEFCFDBF0DBAD03D0010EDA6F01D07F
:100C1000DA6BDA2D03D0C80EDB6F02D0880EDB6FE3
:100C2000D9B1DB81D9B3DB83DE6BD7C0DDF0E06BFC
:100C3000080EDF6F71EC01F002C0DDF001C0DCF0E6
:100C4000040EDC27000EDD23DCC0E9FF040EDD25E9
:100C5000EA6EDBC0EFFF010E016E03D000D0000E84
:100C6000016E000C9851010A03E0030A13E024D03E
:100C7000EA6A4A0EE96E040EE26E180EE16E080E84
:100C8000016EE6CFEEFF012EFCD7D16BFDEC01F03B
:100C9000986B14D0EA6A410EE96E040EE26E180EEB
:100CA000E16E070E016EE6CFEEFF012EFCD7986BCA
:100CB000D16BFDEC01F002D0986B00D094EF06F000
:100CC000DE6BCFC0DDF0E06B080EDF6F71EC01F082
:100CD00002C0D1F001C0D0F0010E0124016E000E5F
:100CE0000220036E01C0E9FF040E0324EA6E036ACA
:100CF000EFCF01F003C002F08AEF06F09291020EEE
:100D0000CF6FD06F94DE8FEF06F09281946B020E5E
:100D1000CF6FD6D701C093F0935301E1EFD799EF8E
:100D200006F0CE5302E19ED704D0CE51020801E175
:100D3000ECD7000CCFC06EFFCF5303E0040E3A6E29
:100D400002D0020E3A6EAAEF06F0336A326A3CC055
:100D5000CFF0F0D719EF07F0CFC0DCF0D7DE0152AB
:100D600046E0DE6BCFC0DDF0E06B080EDF6F71ECAC
:100D700001F002C0D8F001C0D7F0040ED727000E52
:100D8000D823020ED725016E000ED821036E01C0B4
:100D9000E9FF040E0324EA6EECCF03F0ED52EFCF2F
:100DA000D5F003C0D6F0D6C0EAFFD5C0E9FFD1C068
:100DB000E2FFD0C0E1FFD3C002F0D2C001F0015287
:100DC00002E0022A02D0025206E0E6CFEEFF012E38
:100DD000FCD7022EFAD7CFC0D7F0D3C0D9F0D2C0FB
:100DE000D8F0D4C0DAF0B9DE015003D000D0000E44
:100DF000016E000C020ECF6FD16B520ED06FD36B11
:100E000091C0D2F0020ED46FA7DF91C097F0916B22
:100E1000000C915301E0EEDF1EEF07F0CE530AE124
:100E2000322C03D003EC02F004D03250020801E16E
:100E30008CD704D0CE51020801E1EBD7000C393039
:100E4000CC6FCC33CC331F0ECC17395242E10401A6
:100E500000513C0B0001CD6F430E0401001700014F
:100E6000CD5134081EE104010451800B01E0046BF4
:100E70000001C3D56D983B3C05D0CF6B030ED06FFE
:100E8000D6DD0ED0CF6B020ED06FD1DD3B50FE0809
:100E900007E0D76BD96B3BC0D8F0040EDA6F5DDE8C
:100EA00017D0CD51040814E1CE6B3BDFCF6B020E9F
:100EB000D06FBDDD3B50FE080AE03B3C01D007D0BF
:100EC000D76BD96B3BC0D8F0010EDA6F46DE00D08D
:100ED0007AD03950040814E1430E04010417FF0EC0
:100EE0003B6E0001CE6B9ADF3B3C01D008D0D76B44
:100EF000D96B3BC0D8F0020EDA6F2FDE00D063D082
:100F000039B42AD0DE6BCCC0DDF0E06B080EDF6FA9
:100F100071EC01F001C0CEF001C001F0040E02241A
:100F2000036E01C0CEF0CF6FDE6BCCC0DDF0E06BA6
:100F3000080EDF6F71EC01F001C0E9FF040E02241E
:100F4000EA6EEF50430BCFC0EAFFCEC0E9FFEF6E71
:100F5000CCC0CEF0E6DE37D0DE6BCCC0DDF0E06B8F
:100F6000080EDF6F71EC01F002C0CFF001C0CEF0CF
:100F7000040ECE27000ECF23CEC001F0040ECF25E5
:100F8000036ECEC0CEF0CF6FDE6BCCC0DDF0E06B79
:100F9000080EDF6F71EC01F002C0D1F001C0D0F09B
:100FA000040ED027000ED123D0C0E9FF040ED125B6
:100FB000EA6EEF50430BCFC0EAFFCEC0E9FFEF6E01
:100FC000CCC0CEF02BDF1CEF08F0A19A3A5201E121
:100FD00039D0685237E068A404D069A402D02CEF5D
:100FE00001F06DA201D02ED068AA04D069AA02D067
:100FF00044EF01F068A204D069A202D04BEF01F0E7
:1010000068A004D069A002D0E0EF01F068A804D085
:1010100069A802D0F5EF01F068AC04D069AC02D049
:10102000FAEF01F0CB6B68A608D069A606D06CCFAA
:1010300039F002EC00F003D701D004D0CB51CB2B18
:101040000308F1E236EF00F00C2053544F505741A3
:101050005443483031410000204B616B6C696B2078
:101060003230313000000C57616974696E67206658
:101070006F722050432E2E2E20000C2050432063F0
:101080006F6E6E65637465642E2E2E000C0A5354C9
:101090004152542020202020202054455354000049
:1010A0000C0A2020202020202020455343000C0A39
:1010B0005354415254202020202020205445535482
:1010C00000000C0A20202053544F5000EA6AA40E5E
:1010D000E96EEF500EE0070E016E006A002EFED79B
:1010E000012EFBD7C70E006E002EFED70000EF2E9C
:1010F000F2D7000CABB102D08C9801D08C889598B7
:10110000ABB302D08C9A01D08C8A959AABB502D041
:101110008C9C01D08C8C959CABB702D08C9E01D05E
:101120008C8E959E00008D809690030E006E002E92
:10113000FED700D08D909690000CAC6B9588000E79
:1011400083B8010EAC13958A000E83BA010E006EAF
:10115000D89000360050AC13958C000E83BC010E65
:10116000006E00360036FC0E00160050AC13958E53
:10117000000E83BE010E006E003600360036F80EFB
:1011800000160050AC13ACC001F0000C9588958A95
:10119000958C958E8D84969400008D80969000009D
:1011A000CCDF01C0ABF08D90969000008D809690C2
:1011B00000D000D000D0C1DF01C0AAF08D90969081
:1011C0009598959A959C959EAB39006EF00E0016F9
:1011D0000050AA11016EF3EF08F096909692969443
:1011E0008D929692D3D701C0AAF001BEFBD7A85327
:1011F00002E18D9201D08D82969200008D9496949A
:1012000000008D909690A939AA6F0F0EAA17AAC058
:10121000ABF070DFA9510F0BAA6FAB6F6BDF000C47
:101220009598959A959C959E9690969296948D9267
:1012300096928D9496948D9096900F0EA46F46DFA3
:10124000010E996F9951030808E3030EAB6F52DF4B
:10125000050EA46F3BDF992BF5D7020EAB6F4ADF6B
:10126000996B995103080AE3036A99515DEC00F008
:101270009A6FA86BA96FB1DF992BF3D76FEF0DF0C1
:101280006D6A696A080E6F6E94503009946E3A6AFE
:10129000196AF2BE198EF29ECCEC01F019BEF28EE4
:1012A00053EF09F0EDD779EF09F0196AF2BE198E04
:1012B000F29ECCEC01F019BEF28E6D6A140E6F6EC8
:1012C000696A6D86010E3A6E69EF09F06DB601D05C
:1012D000ECD73A2C0BD06DBA09D0686A696AA08A3B
:1012E000C00EF212110E696E020E3A6E7AEF09F01C
:1012F000D9D7ECD73A500208FCE170EF0DF0A52DDC
:1013000001D003D0400EA66F01D0A66B010EA45DE4
:10131000A627A6518009A76FA86BA96F5EDF000CF6
:10132000A351070A07E00B0A0AE0060A10E0020AC6
:1013300014E018D0010EA46FA56FE1DF19D0A86BDF
:10134000010EA96F4ADF020EA46FC0DE11D0010E9C
:10135000A46F020EA56FD3DF0BD0A86B100EA96F80
:101360003CDF06D0010EA86FA3C0A9F036DF00D085
:10137000000C0900F5520CE0F6CF99F0F7CF9AF087
:10138000F5CFA3F0CDDF99C0F6FF9AC0F7FFF1D7F4
:10139000000C030E9C5F0AE3EA6A9C0EE96EEF50B4
:1013A00005E002D000D00000EF2EFCD7E2EF09F0FC
:1013B00099519A110EE094908B70040E9B6FC80E99
:1013C0009C6FE7D79B2FFBD79951D8B49A07990701
:1013D000EFD79BEF0DF0A451016AA35D03E2A3C018
:1013E00000F00CD0006A080EA56FA3370036A45198
:1013F000005CD8B0006E0136A52FF7D7000C015065
:10140000A1C0A3F0640EA46FE6DF00C0A1F00150FC
:10141000300E07E1A2A30CD0A2B70AD0A2B9200EC9
:1014200003D0A297A299A281012601C0A3F078DF80
:10143000A1C0A3F00A0EA46FCEDF00C0A1F001503E
:10144000300E06E1A2B708D0A2A106D0A2B9200EA4
:10145000012601C0A3F064DF300EA127A1C0A3F0D4
:101460005FDF000CB60E006E036A026A016AA551C6
:10147000A611A711A81102E1006A0DD0D89001BEF3
:1014800009D0A537A637A737A83703360236013665
:10149000002EF4D7019E000CA551D8B4A5D0B16F91
:1014A000A951D8B4A1D0B15F05E37F0EB127D8B060
:1014B0009BD006D0810EB15FD8A096D0D8B494D07E
:1014C000B1C000F0016A026A036AB06BA6C0AFF057
:1014D000AF8FA7C0AEF0A8C0ADF0190EB16FAC5180
:1014E000AD5F0DE2010EAE5F0AE2AF5F08E2B05FF2
:1014F00006E2B02BAF2BAE2BAC51AD2728D0AB51B1
:10150000AE5F12E2010EAF5F0FE2B05F0DE2B02BF3
:10151000AF2BAB51AE27AC51AD2719E3AE2B17E182
:10152000AF2B15E1B02B13D0AA518009AF5F0EE2AB
:10153000010EB05F0BE2B02BAA518009AF27AB516F
:10154000AE27E9E3AF2BE7E1B02BE5D70380B12F5E
:1015500001D00BD0D890AD37AE37AF37B037D89079
:10156000033602360136B237BAD7B2A106D0D890C8
:10157000013202320332B23302D0000635E0B2BF8C
:101580001ED0D890AD37AE37AF37B037AC51AD5F66
:1015900007E2010EAE5F04E2AF5F02E2B05F1AE362
:1015A000AB51AE5F05E2010EAF5F02E2B05F12E346
:1015B000AA518009AF5F03E2010EB05F0BE3032A7B
:1015C00009E1022A07E1012A05E1002A0DE00132C2
:1015D00002320332A6C0B1F0AA51B11BB1AF02D0A2
:1015E000018E06D0019E04D0006A016A026A036A75
:1015F000000CB991F2BEB981F29E91513E0802E20F
:101600003E0E916F9151912B036A520FE96E000EBD
:101610000320EA6EB8C0EFFFF29EB9B1F28E14EF6C
:101620000BF0B7C0B8F0E5D7196AF2BE198EF29E7A
:10163000020EDC6F86EC05F019BEF28E015208E056
:10164000196AF2BE198EF29EFAEC06F019BEF28EFD
:1016500045EF0BF091513E0815E2196AF2BE198E62
:10166000F29E020EDC6F86EC05F019BEF28E01527E
:1016700008E0196AF2BE198EF29EFAEC06F019BE65
:10168000F28EE8D7B6C0B7F0CCD7000C006A016A7A
:10169000026A036ABE6BBF6BC06BC16BBD51BC11EC
:1016A000BB11BA112CE0200EC26FD890B637B737F5
:1016B000B837B937BE37BF37C037C137BD51C15D45
:1016C00008E1BC51C05D05E1BB51BF5D02E1BA510B
:1016D000BE5D0FE3BA51BE5FBB51D8A0BB3DBF5F3B
:1016E000BC51D8A0BC3DC05FBD51D8A0BD3DC15FBD
:1016F000D8800036013602360336C22FD6D7EA6AC2
:10170000BE0EE96E000CE950AD6F3B0EB46F9A0E41
:10171000B36FCA0EB26FB16B0A0EAF6FACC0B9F047
:10172000ABC0B8F0AAC0B7F0A9C0B6F0B4C0BDF065
:10173000B3C0BCF0B2C0BBF0B1C0BAF0A7DF01507B
:10174000EFCFA9F0ECCFAAF0ECCFABF0ECCFACF040
:1017500000520FE1AF51010A0CE0AD510BE00F0B4D
:10176000AF5D01E00CE2ADBF0AD0ADBD03D0200EED
:1017700002D0AD6B300E002600C0B6F06BDFB4C0F7
:10178000B9F0B3C0B8F0B2C0B7F0B1C0B6F0BD6B3D
:10179000BC6BBB6B0A0EBA6F79DF03C0B4F002C03A
:1017A000B3F001C0B2F000C0B1F0AF2FB7D795EFE2
:1017B0000FF0B651D8B471D0006EBA51D8B46DD014
:1017C000002604E3810E002668E204D07F0E005E4E
:1017D00064E363E0B7C0BEF0BB51BE1BB78FBB8FE5
:1017E000B951BD03F4CFC0F0B851BC03F4CF03F03E
:1017F000F3CFBFF0BD03F350C027F450BF23000E5A
:101800000322B951BC03F350C027F450BF23000E8C
:10181000026A03220222B751BD03F350BF27F450DE
:101820000322000E0222B751BC03F3500326F450EA
:101830000222000E016A0122B951BB03F350BF27F7
:10184000F4500322000E02220122B851BB03F350D0
:101850000326F4500222000E0122B751BB03F350BD
:101860000226F4500122002A01BE05D0BF370336FC
:10187000023601360006000EBFAF0AD0032A02224C
:101880000122015005E1025003E1035001E1002A69
:10189000BEBF018EBEAF019E04D0006A016A026A1B
:1018A000036A87EF0CF0B651B608B66F036AB7C08B
:1018B000BAF0B78FD890B733B833B93303320232A6
:1018C00001320032B62FF6D7BAAF0BD0001E011E80
:1018D000021E031E002AD8B4012AD8B4022AD8B4A2
:1018E000032A9AEF0CF0E950AE6FAD51B06F19E0DA
:1018F000ACC0B9F0ABC0B8F0AAC0B7F0A9C0B6F0A0
:10190000BD6BBC6B200EBB6F820EBA6F52D703C08B
:10191000ACF002C0ABF001C0AAF000C0A9F0B02F3B
:10192000E7D7ACC0B9F0ABC0B8F0AAC0B7F0A9C057
:10193000B6F0B9D703C0ACF002C0ABF001C0AAF05A
:1019400000C0A9F0ACAF0DD0AE07AE8BA91FAA1F87
:10195000AB1FAC1FA92BD8B4AA2BD8B4AB2BD8B4CF
:10196000AC2B3B0EB56F9A0EB46FCA0EB36FB26B51
:101970000A0EB06FAD51D8B4AE2BACC0B9F0ABC04D
:10198000B8F0AAC0B7F0A9C0B6F0B5C0BDF0B4C0F9
:10199000BCF0B3C0BBF0B2C0BAF078DE0150EFCFFC
:1019A000A9F0ECCFAAF0ECCFABF0ECCFACF000524A
:1019B0000FE1AD29B05D0CE0AE510CE00F0BB05D56
:1019C00001E037E2AEBF35D0AEBD04D0200E2DD041
:1019D000200EAE17AEAB0CD0AE9BAD51D8A4AE0767
:1019E0000050AE6F2D0EB66F35DEAE51006EAE6B91
:1019F000AD51B05D0AE10050AE6F2E0EB66F2ADE1B
:101A0000AE51006E200EAE17000E300EAEAB0DD0F4
:101A1000AE9BAD51D8A4AE070050AE6F2D0EB66F81
:101A200019DEAE51006EAE6B300E002600C0B6F06F
:101A300011DEB5C0B9F0B4C0B8F0B3C0B7F0B2C0F1
:101A4000B6F0BD6BBC6BBB6B0A0EBA6F1FDE03C07A
:101A5000B5F002C0B4F001C0B3F000C0B2F0B02FD6
:101A60008CD7000CF86AD09E078EEA6AE96A3A6A57
:101A70003E6A916B986BC150C00B0F09C16E070E87
:101A8000B46E366A040E376E0C0E386EC150C00B41
:101A90000F09C16EF19EC2909698C69A949E93804B
:101AA0009392010EC66E000EC76ED190870ED56E52
:101AB000CD6A000ECA6E000ECB6EB16A070EB46E10
:101AC0009250926E130E006E002EFED700D0B450CE
:101AD000A19CB56AF28AC00EF21210EF09F008D488
:101AE000010EA46FA56F0BDC480EF66E100EF76E9C
:101AF00040DC010EA46F020EA56F01DC580EF66EDD
:101B0000100EF76E36DC040E996FFA0EA46F66ECB9
:101B100008F0992FFAD7660EF66E100EF76E29DCD4
:101B200095A1FED77A0EF66E100EF76E22DC9A6B38
:101B30000A0E996F3DD4316A306A2F6A2E6A95A1D8
:101B400039D2010E2E26D8B02F2AD8B4302AD8B4D4
:101B5000312A1D6A1C6A1B6A1A6A216A206A1F6A76
:101B60001E6A256A246A236A226A296A286A276A01
:101B7000266A8C0EF66E100EF76EB9EC09F09580A1
:101B800083A091D0958683B68DD0A00EF66E100EF0
:101B9000F76EB9EC09F0958483A47ED0010EA46F92
:101BA000A56F7FEC09F09380000E81B0010E996F54
:101BB0009382000E81B2010E9A6F9384000E81B45D
:101BC000010E9B6F9386000E81B6010E9C6F938869
:101BD000000E81B8010E9D6F938A000E81BA010E2E
:101BE0009E6F938C000E81BC010E9F6F938E000E32
:101BF00081BE010EA06F99C0A1F0180EA26FFFEC7C
:101C000009F0200EA36F90EC09F09AC0A1F0180E15
:101C1000A26FFFEC09F0200EA36F90EC09F09BC0BF
:101C2000A1F0180EA26FFFEC09F0200EA36F90EC4C
:101C300009F09CC0A1F0180EA26FFFEC09F0200E75
:101C4000A36F90EC09F09DC0A1F0180EA26FFFECFD
:101C500009F0200EA36F90EC09F09EC0A1F0180EC1
:101C6000A26FFFEC09F0200EA36F90EC09F09FC06B
:101C7000A1F0180EA26FFFEC09F0200EA36F90ECFC
:101C800009F0A0C0A1F0180EA26FFFEC09F0640EDD
:101C9000A46F66EC08F07FD7AE0EF66E100EF76EEE
:101CA000B9EC09F06CD7C20EF66E100EF76EB9ECF7
:101CB00009F0938081B003D0958283B2FAD72D6A60
:101CC0002C6A2B6A2A6AD76AD66A938281B218D0A4
:101CD000958283A215D02BC09DF02AC09CF09A6BF0
:101CE0009B6BD650D7CF03F09A251A6ED7509B2105
:101CF0001B6E000E2A201C6E000E2B201D6EE5D7D9
:101D0000938481B403D0958283B2FAD72D6A2C6A6A
:101D10002B6A2A6AD76AD66A938681B618D09582CA
:101D200083A215D02BC09DF02AC09CF09A6B9B6BB0
:101D3000D650D7CF03F09A251E6ED7509B211F6E29
:101D4000000E2A20206E000E2B20216EE5D79388EE
:101D500081B803D0958283B2FAD72D6A2C6A2B6A98
:101D60002A6AD76AD66A938A81BA18D0958283A2E2
:101D700015D02BC09DF02AC09CF09A6B9B6BD6505F
:101D8000D7CF03F09A25226ED7509B21236E000EE9
:101D90002A20246E000E2B20256EE5D7938C81BC63
:101DA00003D0958283B2FAD72D6A2C6A2B6A2A6AED
:101DB000D76AD66A938E81BE18D0958283A215D039
:101DC0002BC09DF02AC09CF09A6B9B6BD650D7CF4E
:101DD00003F09A25266ED7509B21276E000E2A20ED
:101DE000286E000E2B20296EE5D71DC0A8F01CC060
:101DF000A7F01BC0A6F01AC0A5F032EC0AF003C091
:101E0000A8F002C0A7F001C0A6F000C0A5F0AC6B1E
:101E1000AB6B7A0EAA6F820EA96F4CEC0AF000C071
:101E200099F001C09AF002C09BF003C09CF021C061
:101E3000A8F020C0A7F01FC0A6F01EC0A5F032EC8D
:101E40000AF003C0A8F002C0A7F001C0A6F000C0CD
:101E5000A5F0AC6BAB6B7A0EAA6F820EA96F4CEC3F
:101E60000AF000C09DF001C09EF002C09FF003C0C8
:101E7000A0F025C0A8F024C0A7F023C0A6F022C07F
:101E8000A5F032EC0AF003C0A8F002C0A7F001C030
:101E9000A6F000C0A5F0AC6BAB6B7A0EAA6F820EF9
:101EA000A96F4CEC0AF000C0A1F001C0A2F002C082
:101EB000A3F003C0A4F029C0A8F028C0A7F027C051
:101EC000A6F026C0A5F032EC0AF003C0A8F002C0CC
:101ED000A7F001C0A6F000C0A5F0AC6BAB6B7A0E0A
:101EE000AA6F820EA96F4CEC0AF000C0A5F001C0E9
:101EF000A6F002C0A7F003C0A8F00A0EB66F2AEC45
:101F00000BF00D0EB66F2AEC0BF0200EB66F2AEC1C
:101F10000BF0070EE96E31C0ACF030C0ABF02FC053
:101F2000AAF02EC0A9F083EF0BF0200EB66F2AECBA
:101F30000BF0060EE96E9CC0ACF09BC0ABF09AC0F3
:101F4000AAF099C0A9F0010EAD6FCDDC200EB66FDE
:101F50002AEC0BF0060EE96EA0C0ACF09FC0ABF00F
:101F60009EC0AAF09DC0A9F0010EAD6FBCDC200E92
:101F7000B66F2AEC0BF0060EE96EA4C0ACF0A3C05D
:101F8000ABF0A2C0AAF0A1C0A9F0010EAD6FABDC0E
:101F9000200EB66F2AEC0BF0060EE96EA8C0ACF06E
:101FA000A7C0ABF0A6C0AAF0A5C0A9F0010EAD6F06
:081FB0009ADCC5D5B0D5030091
:020000040030CA
:0E0000003CCE390E0005A1000FC00FE00F40EE
:00000001FF
